:020000040000FA
:04080000B5EF07F059
:1008100003B210EF05F0F2B42BEF05F09EB033EF0A
:1008200005F09EB23BEF05F0F2A81AEF04F0F2B229
:1008300025EF04F0F2A620EF04F0F2B022EF04F06E
:1008400093EF07F0F296F290FF00CD90F2929EA007
:100850002FEF04F00101533F2FEF04F0542BAEC1F2
:10086000B2F1AFC1B3F1B0C1B4F1B1C1B5F1AAC138
:10087000AEF1ABC1AFF1ACC1B0F1ADC1B1F1A6C148
:10088000AAF1A7C1ABF1A8C1ACF1A9C1ADF1A2C158
:10089000A6F1A3C1A7F1A4C1A8F1A5C1A9F19EC168
:1008A000A2F19FC1A3F1A0C1A4F1A1C1A5F19AC178
:1008B0009EF19BC19FF19CC1A0F19DC1A1F196C188
:1008C0009AF197C19BF198C19CF199C19DF1CECF4E
:1008D00096F1CFCF97F153C198F154C199F1CF6AF6
:1008E000CE6A0101536B546B9E90CD800EBC0E8E70
:1008F0000EBA7EEF04F00E8A93EF07F00E8C0EBE58
:10090000BAEF04F096C19AF197C19BF198C19CF19E
:1009100099C19DF19AC19EF19BC19FF19CC1A0F12B
:100920009DC1A1F19EC1A2F19FC1A3F1A0C1A4F1FB
:10093000A1C1A5F1A2C1A6F1A3C1A7F1A4C1A8F1CB
:10094000A5C1A9F1A6C1AAF1A7C1ABF1A8C1ACF19B
:10095000A9C1ADF1AAC1AEF1ABC1AFF1ACC1B0F16B
:10096000ADC1B1F1AEC1B2F1AFC1B3F1B0C1B4F13B
:10097000B1C1B5F101015E6B5F6B606B616B96514C
:100980005E2797515F2398516023995161239A51B3
:100990005E279B515F239C5160239D5161239E5193
:1009A0005E279F515F23A0516023A1516123A25173
:1009B0005E27A3515F23A4516023A5516123A65153
:1009C0005E27A7515F23A8516023A9516123AA5133
:1009D0005E27AB515F23AC516023AD516123AE5113
:1009E0005E27AF515F23B0516023B1516123B251F3
:1009F0005E27B3515F23B4516023B5516123D89072
:100A0000613360335F335E33D890613360335F337B
:100A10005E33D890613360335F335E3393EF07F01A
:100A20000392030103EE00F080517F0BE92604C01E
:100A3000EFFF802B8151805D700BD8A48B8200006A
:100A40008051815D700BD8A48B9281518019D8B4EC
:100A5000079093EF07F0F2940101453F93EF07F001
:100A6000462B93EF07F09E900101533F93EF07F061
:100A7000542B93EF07F09E9204005CA140EF05F029
:100A8000077C07AC5BEF05F0C274C2B455EF05F00C
:100A9000C3CFADF5C4CFAEF50501D890AE33AD33BD
:100AA000D890AE33AD335CEF05F0C3CF55F1C4CF72
:100AB00056F15CEF05F0C28207B4C9EF05F047C1FB
:100AC0004BF148C14CF149C14DF14AC14EF15EC1F3
:100AD00062F15FC163F160C164F161C165F196C10A
:100AE000B6F197C1B7F198C1B8F199C1B9F19AC1FE
:100AF000BAF19BC1BBF19CC1BCF19DC1BDF19EC1CE
:100B0000BEF19FC1BFF1A0C1C0F1A1C1C1F1A2C19D
:100B1000C2F1A3C1C3F1A4C1C4F1A5C1C5F1A6C16D
:100B2000C6F1A7C1C7F1A8C1C8F1A9C1C9F1AAC13D
:100B3000CAF1ABC1CBF1ACC1CCF1ADC1CDF1AEC10D
:100B4000CEF1AFC1CFF1B0C1D0F1B1C1D1F1B2C1DD
:100B5000D2F1B3C1D3F1B4C1D4F1B5C1D5F1ADC5B2
:100B6000AFF5AEC5B0F5AFC5B1F5B0C5B2F5010191
:100B700055515B2756515C23E86A5D230D2EC9EF62
:100B800005F05CC157F15DC158F15B6B5C6B5D6B4F
:100B9000078E0201002F93EF07F03C0E006F00C19B
:100BA0000CF101C10DF102C10EF103C10FF104C13D
:100BB00010F105C111F106C112F107C113F108C10D
:100BC00014F109C115F10AC116F10BC117F134C1B5
:100BD00035F105012951000AD8B492EF06F005015C
:100BE0002951010AD8B41CEF06F005012951020A67
:100BF000D8B45DEF06F005012951030AD8B45DEFC2
:100C000006F005012951040AD8B45DEF06F005018C
:100C10002951050AD8B45DEF06F005012951060AED
:100C2000D8B45DEF06F005012951070AD8B45DEF8D
:100C300006F0296B92EF06F005014D6727EF06F0ED
:100C40004E6727EF06F04F6727EF06F050672BEF50
:100C500006F092EF06F051C500F152C501F153C5FF
:100C600002F154C503F10101010E046F000E056F7E
:100C7000000E066F000E076F6BEC1CF000C151F503
:100C800001C152F502C153F503C154F5006750EF9D
:100C900006F0016750EF06F0026750EF06F00367B9
:100CA00092EF06F04DC551F54EC552F54FC553F5BF
:100CB00050C554F50E8892EF06F005012A6763EFE0
:100CC00006F092EF06F00EBE78EF06F00FA07DEF73
:100CD00006F00101476774EF06F0486774EF06F00D
:100CE000496774EF06F04A6778EF06F07DEF06F08B
:100CF00007AE7DEF06F08FEF06F005012B2F92EF88
:100D000006F03C0E2B6F2A2F92EF06F00101000E29
:100D1000626FE00E636FA50E646F010E656F0501D3
:100D20002A6B0E8805015C6B2DB798EF06F05C818D
:100D30000CC100F10DC101F10EC102F10FC103F1AF
:100D400010C104F111C105F112C106F113C107F17F
:100D500014C108F115C109F116C10AF117C10BF14F
:100D600035C134F100C10CF101C10DF102C10EF128
:100D700003C10FF104C110F105C111F106C112F157
:100D800007C113F108C114F109C115F10AC116F127
:100D90000BC117F134C135F101018A67D7EF06F0B5
:100DA0008B67D7EF06F08C67D7EF06F08D67DBEF28
:100DB00006F00BEF07F08EC100F18FC101F190C179
:100DC00002F191C103F10101010E046F000E056FE4
:100DD000000E066F000E076F6BEC1CF000C18EF169
:100DE00001C18FF102C190F103C191F1006700EFE1
:100DF00007F0016700EF07F0026700EF07F00367F5
:100E00000BEF07F08AC18EF18BC18FF18CC190F18D
:100E10008DC191F10E80D57ED5BE69D0D6CF47F178
:100E2000D7CF48F145C149F1E86AE8CF4AF10F90C0
:100E300047C100F148C101F149C102F14AC103F1C2
:100E400001010A0E046F000E056F000E066F000E02
:100E5000076F6BEC1CF000AF0F80010154A73DEF52
:100E600007F00E9A0E9C0E9E0101000E5E6F600E42
:100E70005F6F3D0E606F080E616F010147BF4DEF60
:100E800007F048674DEF07F049674DEF07F04A67F5
:100E90004DEF07F0F28872EF07F0F2985E6B5F6B30
:100EA000606B616B966B976B986B996B9A6B9B6B96
:100EB0009C6B9D6B9E6B9F6BA06BA16BA26BA36BDE
:100EC000A46BA56BA66BA76BA86BA96BAA6BAB6B8E
:100ED000AC6BAD6BAE6BAF6BB06BB16BB26BB36B3E
:100EE000B46BB56BD76AD66A0101456B466B0CC112
:100EF00000F10DC101F10EC102F10FC103F110C1EA
:100F000004F111C105F112C106F113C107F114C1B9
:100F100008F115C109F116C10AF117C10BF135C16C
:100F200034F193EF07F002C0E0FF005001C0D8FF9A
:100F30001000A6B299EF07F00CC0A9FF0BC0A8FFE4
:100F4000A69EA69CA684F29E550EA76EAA0EA76E1C
:100F5000A682F28EA694A6B2ABEF07F01200A96E9D
:100F6000A69EA69CA680A8501200076A0E6A0F6A69
:100F70000F010D0EC16E860EC06E030EC26E0F0104
:100F8000280E896E130E926E080E8A6EF30E936E03
:100F90008B6A900E946EF18EF19E0D6A01015B6B6F
:100FA0005C6B5D6B576B586BF29A0101476B486B3A
:100FB000496B4A6B4B6B4C6B4D6B4E6B4F6B506B75
:100FC000516B526B456B466BD76AD66A0F01280E80
:100FD000D56EF28A9D90B00ECD6E01015E6B5F6B97
:100FE000606B616B626B636B646B656B666B676B8D
:100FF000686B696B536B546BCF6ACE6A0E9A0E9C0A
:101000000E9E9D80760ECA6E9D8202013C0E006F80
:10101000CC6A160EAFEC07F0E8CF00F1170EAFEC7C
:1010200007F0E8CF01F1180EAFEC07F0E8CF02F1BE
:10103000190EAFEC07F0E8CF03F1010103AF3BEF6E
:1010400008F062EC1DF0160E0C6E00C10BF099EC6E
:1010500007F0170E0C6E01C10BF099EC07F0180E9B
:101060000C6E02C10BF099EC07F0190E0C6E03C167
:101070000BF099EC07F000C18AF101C18BF102C1BC
:101080008CF103C18DF100C18EF101C18FF102C15C
:1010900090F103C191F11A0EAFEC07F0E8CF00F127
:1010A0001B0EAFEC07F0E8CF01F11C0EAFEC07F020
:1010B000E8CF02F11D0EAFEC07F0E8CF03F101011C
:1010C00003AF91EF08F062EC1DF01A0E0C6E00C138
:1010D0000BF099EC07F01B0E0C6E01C10BF099ECB4
:1010E00007F01C0E0C6E02C10BF099EC07F01D0E00
:1010F0000C6E03C10BF099EC07F01A0EAFEC07F081
:10110000E8CF00F11B0EAFEC07F0E8CF01F11C0EA9
:10111000AFEC07F0E8CF02F11D0EAFEC07F0E8CF1F
:1011200003F100C192F101C193F102C194F103C135
:1011300095F1240EAC6E900EAB6E240EAC6E080EC4
:10114000B86E000EB06E1F0EAF6E0401806B816B27
:101150000F01900EAB6E0F019D8A0301806B816BB6
:10116000A26B8B9286EC20F0200EAFEC07F0E8CF5C
:1011700029F505012951FF0AD8A4C6EF08F0296B0B
:10118000200E0C6E29C50BF099EC07F00501010E3D
:101190002A6F3C0E2B6F250EAFEC07F0E8CF00F165
:1011A000260EAFEC07F0E8CF01F1270EAFEC07F009
:1011B000E8CF02F1280EAFEC07F0E8CF03F1010110
:1011C00003AFFDEF08F062EC1DF0250E0C6E00C1C0
:1011D0000BF099EC07F0260E0C6E01C10BF099ECA8
:1011E00007F0270E0C6E02C10BF099EC07F0280EE9
:1011F0000C6E03C10BF099EC07F000C14DF501C175
:101200004EF502C14FF503C150F500C151F501C1C2
:1012100052F502C153F503C154F5290EAFEC07F0A6
:10122000E8CF55F505015651555DD8A055C556F581
:1012300005012951020A0EE181B82AEF09F00501E2
:10124000562F27EF09F055C556F52AEF09F081BA58
:10125000A5EF23F0210EAFEC07F0E8CF00F1220E4E
:10126000AFEC07F0E8CF01F1230EAFEC07F0E8CFC9
:1012700002F1240EAFEC07F0E8CF03F1010103AF58
:1012800070EF09F062EC1DF0210E0C6E00C10BF046
:1012900099EC07F0220E0C6E01C10BF099EC07F0EF
:1012A000230E0C6E02C10BF099EC07F0240E0C6EAD
:1012B00003C10BF099EC07F0210EAFEC07F0E8CF7B
:1012C00000F1220EAFEC07F0E8CF01F1230EAFECF6
:1012D00007F0E8CF02F1240EAFEC07F0E8CF03F1FE
:1012E00000C157F501C158F502C159F503C15AF5BE
:1012F000BDEC1FF07FEC1EF0CFEC1DF00501295175
:10130000030A12E005012951040A1DE005012951D3
:10131000050A24E005012951060A32E00501295198
:10132000070A38E0D3EF09F0A6C500F101010F0E5E
:10133000001701010051000A36E001010051050AC1
:1013400032E0D0EF09F0A6C500F101010F0E001741
:1013500001010051000A27E0D0EF09F00501A65174
:10136000000A21E00501A651150A1DE00501A6515C
:10137000300A19E00501A651450A15E0D0EF09F041
:101380000501A651000A0FE00501A651300A0BE045
:10139000D0EF09F00501A651000A05E0D0EF09F0F1
:1013A00081BAA5EF23F007900001F28EF28C07B00E
:1013B00003EF1AF00EB0E4EF14F00EB8D6EF0EF013
:1013C0000301805181197F0BD8B403EF1AF013EE9B
:1013D00000F081517F0BE126812BE7CFE8FFE00B86
:1013E000D8B403EF1AF023EE82F0A2511F0BD926D6
:1013F000E7CFDFFFA22BDF50780AD8A403EF1AF063
:1014000007808EC100F18FC101F190C102F191C13D
:1014100003F10101040E046F000E056F000E066F4C
:10142000000E076F6BEC1CF000AF20EF0AF001011B
:10143000030E8E6F000E8F6F000E906F000E916F77
:1014400003018251720AD8B4E4EF14F08251520AB7
:10145000D8B4E4EF14F08251750AD8B4E4EF14F074
:101460008251630AD8B4BFEF16F08251690AD8B42A
:101470009FEF11F082517A0AD8B4B2EF12F0825184
:10148000490AD8B43EEF11F08251500AD8B45CEF4B
:1014900010F08251700AD8B49FEF10F08251540AB4
:1014A000D8B4CAEF10F08251740AD8B410EF11F01A
:1014B0008251730AD8B414EF14F08251530AD8B48D
:1014C00079EF14F082514C0AD8B47CEF0AF0F4EFB3
:1014D00016F0040114EE00F080517F0BE12682C467
:1014E000E7FF802B12000D0E826F69EC0AF00A0EE6
:1014F000826F69EC0AF0120003018351300AD8B4FC
:101500002BEF0DF003018351310AD8B4B1EF0DF088
:1015100003018351320AD8B401EF0EF00301835165
:10152000330AD8B405EF0EF003018351340AD8B45E
:1015300013EF0EF003018351350AD8B4DBEF0EF040
:10154000030183514D0AD8B4A4EF0BF0030183517A
:101550006D0AD8B4BEEF0BF003018351490AD8B429
:10156000DBEF0FF003018351500AD8B40DEF0FF0F9
:1015700003018351540AD8B486EF0FF0030183515D
:10158000630AD8B4DEEF0BF003018351430AD8B4E9
:10159000D6EF0CF003018351730AD8B4DCEF0BF0E3
:1015A00003018351610AD8B4F1EF0AF003018351BA
:1015B000650AD8B479EF0DF003018351450AD8B418
:1015C00087EF0DF003018351620AD8B495EF0DF057
:1015D00003018351420AD8B4A3EF0DF0D8A4F4EF6D
:1015E00016F004014C0E826F69EC0AF00401610EE2
:1015F000826F69EC0AF07FEC1EF004012C0E826F02
:1016000069EC0AF062EC1DF0A5C500F1010105ECE2
:101610001DF031C182F40401300E822769EC0AF01A
:1016200032C182F40401300E822769EC0AF033C122
:1016300082F40401300E822769EC0AF004012C0EBA
:10164000826F69EC0AF062EC1DF0A6C500F10101A1
:1016500005EC1DF031C182F40401300E822769ECE3
:101660000AF032C182F40401300E822769EC0AF0DC
:1016700033C182F40401300E822769EC0AF00401C0
:101680002C0E826F69EC0AF062EC1DF0A7C500F128
:10169000010105EC1DF031C182F40401300E8227F6
:1016A00069EC0AF032C182F40401300E822769EC41
:1016B0000AF033C182F40401300E822769EC0AF08B
:1016C00004012C0E826F69EC0AF062EC1DF0A8C5D3
:1016D00000F1010105EC1DF031C182F40401300E6E
:1016E000822769EC0AF032C182F40401300E8227AD
:1016F00069EC0AF033C182F40401300E822769ECF0
:101700000AF004012C0E826F69EC0AF062EC1DF005
:10171000ADC500F1010105EC1DF031C182F40401F9
:10172000300E822769EC0AF032C182F40401300ED7
:10173000822769EC0AF033C182F40401300E82275B
:1017400069EC0AF009EF0FF0A3EC1DF084C333F14C
:10175000B0EC1DF027EC1DF0200E0C6E00C10BF05C
:1017600099EC07F000C129F505012951000A06E0AE
:1017700005012951010A02E025EC1FF004014C0E7D
:10178000826F69EC0AF004014D0E826F69EC0AF079
:1017900004012C0E826F69EC0AF062EC1DF029C581
:1017A00000F105EC1DF033C182F40401300E8227F4
:1017B00069EC0AF009EF0FF0A5EF23F004014C0EDD
:1017C000826F69EC0AF00401630E826F69EC0AF023
:1017D000CFEC1DF004012C0E826F69EC0AF0F3ECE3
:1017E0000BF009EF0FF062EC1DF0ABC500F1010149
:1017F000003B0F0E001705EC1DF033C182F404010D
:10180000300E822769EC0AF0ABC500F101010F0E22
:101810000101001705EC1DF033C182F40401300E04
:10182000822769EC0AF004012D0E826F69EC0AF040
:10183000AAC500F10101003B0F0E001705EC1DF0D9
:1018400033C182F40401300E822769EC0AF0AAC584
:1018500000F101010F0E0101001705EC1DF033C16D
:1018600082F40401300E822769EC0AF004012D0E87
:10187000826F69EC0AF0A9C500F10101003B0F0E6F
:10188000001705EC1DF033C182F40401300E8227ED
:1018900069EC0AF0A9C500F101010F0E0101001762
:1018A00005EC1DF033C182F40401300E822769EC8F
:1018B0000AF00401200E826F69EC0AF0A8C500F15D
:1018C0000F0E0101001705EC1DF033C182F4040175
:1018D000300E822769EC0AF00401200E826F69EC59
:1018E0000AF0A7C500F101010101003B0F0E00172E
:1018F00005EC1DF033C182F40401300E822769EC3F
:101900000AF0A7C500F101010F0E0101001705EC57
:101910001DF033C182F40401300E822769EC0AF015
:1019200004013A0E826F69EC0AF0A6C500F10101CC
:10193000003B0F0E001705EC1DF033C182F40401CB
:10194000300E822769EC0AF0A6C500F101010F0EE6
:101950000101001705EC1DF033C182F40401300EC3
:10196000822769EC0AF004013A0E826F69EC0AF0F2
:10197000A5C500F10101003B0F0E001705EC1DF09D
:1019800033C182F40401300E822769EC0AF0A5C548
:1019900000F101010F0E001705EC1DF033C182F4B8
:1019A0000401300E822769EC0AF0120084C3E8FFBC
:1019B0000F0BE83AE8CFABF585C3E8FF0F0B050145
:1019C000AB1387C3E8FF0F0BE83AE8CFAAF588C34B
:1019D000E8FF0F0B0501AA138AC3E8FF0F0BE83AD3
:1019E000E8CFA9F58BC3E8FF0F0B0501A9138DC341
:1019F000E8FF0F0BE8CFA8F58FC3E8FF0F0BE83A1D
:101A0000E8CFA7F590C3E8FF0F0B0501A71392C31A
:101A1000E8FF0F0BE83AE8CFA6F593C3E8FF0F0BFA
:101A20000501A61395C3E8FF0F0BE83AE8CFA5F52B
:101A300096C3E8FF0F0B0501A5132EEC1EF0040161
:101A40004C0E826F69EC0AF00401430E826F69EC60
:101A50000AF0E8EF0BF066EC23F062EC1DF02DC508
:101A600000F105EC1DF004014C0E826F69EC0AF0E8
:101A70000401300E826F69EC0AF004012C0E826FB3
:101A800069EC0AF031C182F40401300E822769EC5E
:101A90000AF032C182F40401300E822769EC0AF0A8
:101AA00033C182F40401300E822769EC0AF004018C
:101AB0002C0E826F69EC0AF062EC1DF02EC500F16D
:101AC00005EC1DF031C182F40401300E822769EC6F
:101AD0000AF032C182F40401300E822769EC0AF068
:101AE00033C182F40401300E822769EC0AF009EF59
:101AF0000FF004014C0E826F69EC0AF00401650ED0
:101B0000826F69EC0AF00EEC20F009EF0FF004018F
:101B10004C0E826F69EC0AF00401450E826F69EC8D
:101B20000AF02BEC20F009EF0FF004014C0E826F4D
:101B300069EC0AF00401620E826F69EC0AF065EC50
:101B400020F009EF0FF004014C0E826F69EC0AF0EF
:101B50000401420E826F69EC0AF048EC20F009EFB4
:101B60000FF004014C0E826F69EC0AF00401310E93
:101B7000826F69EC0AF004012C0E826F69EC0AF0A6
:101B800025C500F126C501F127C502F128C503F1DD
:101B90000101100E046F000E056F000E066F000E9F
:101BA000076F99EC1CF005EC1DF02EC182F40401C6
:101BB000300E822769EC0AF02FC182F40401300E46
:101BC000822769EC0AF030C182F40401300E8227CA
:101BD00069EC0AF031C182F40401300E822769EC0D
:101BE0000AF032C182F40401300E822769EC0AF057
:101BF00033C182F40401300E822769EC0AF009EF48
:101C00000FF0D0EC20F0F4EF16F004014C0E826FD0
:101C100069EC0AF00401330E826F69EC0AF006ECFD
:101C200021F0BBEF0DF004014C0E826F69EC0AF05D
:101C30000401340E826F69EC0AF004012C0E826FED
:101C400069EC0AF0A3EC1DF084C32AF185C32BF1E3
:101C500086C32CF187C32DF188C32EF189C32FF1E0
:101C60008AC330F18BC331F18CC332F18DC333F1B0
:101C70000101296BB0EC1DF027EC1DF0100E046F74
:101C8000000E056F000E066F000E076F7AEC1CF059
:101C900000C121F501C122F502C123F503C124F5DC
:101CA00019EC23F02EC5A5F52FC5A6F530C5A7F56F
:101CB00031C5A8F532C5A9F533C5AAF534C5ABF5CC
:101CC000F3EC0BF004012C0E826F69EC0AF035C5C1
:101CD00000F136C501F137C502F138C503F1010144
:101CE000000E046F000E056F010E066F000E076FE9
:101CF00099EC1CF005EC1DF0296781EF0EF086EFE2
:101D00000EF004012D0E826F69EC0AF030C182F4EE
:101D10000401300E822769EC0AF031C182F404011B
:101D2000300E822769EC0AF004012E0E826F69ECF6
:101D30000AF032C182F40401300E822769EC0AF005
:101D400033C182F40401300E822769EC0AF00401E9
:101D50002C0E826F69EC0AF062EC1DF039C500F1BF
:101D60003AC501F11EEC18F004012C0E826F69ECEB
:101D70000AF062EC1DF03BC500F105EC1DF031C12D
:101D800082F40401300E822769EC0AF032C182F439
:101D90000401300E822769EC0AF033C182F4040199
:101DA000300E822769EC0AF009EF0FF00E9806EC6E
:101DB00021F009EF0FF004014C0E826F69EC0AF07C
:101DC0000401350E826F69EC0AF004012C0E826F5B
:101DD00069EC0AF062EC1DF00784AFC500F10794CE
:101DE00005EC1DF031C182F40401300E822769EC4C
:101DF0000AF032C182F40401300E822769EC0AF045
:101E000033C182F40401300E822769EC0AF009EF35
:101E10000FF073EC0AF0F4EF16F004014C0E826F31
:101E200069EC0AF00401500E826F69EC0AF00401BB
:101E30002C0E826F69EC0AF085C32AF186C32BF160
:101E400087C32CF188C32DF189C32EF18AC32FF1EA
:101E50008BC330F18CC331F18DC332F18EC333F1BA
:101E60000101B0EC1DF027EC1DF003018451530A71
:101E70000DE0030184514D0A38E00401780E826FB1
:101E800069EC0AF073EC0AF0F4EF16F00401530E5B
:101E9000826F69EC0AF0250E0C6E00C10BF099EC14
:101EA00007F0260E0C6E01C10BF099EC07F0270E1F
:101EB0000C6E02C10BF099EC07F0280E0C6E03C1FA
:101EC0000BF099EC07F000C14DF501C14EF502C1D0
:101ED0004FF503C150F500C151F501C152F502C1E2
:101EE00053F503C154F5EAEF0FF004014D0E826F74
:101EF00069EC0AF0290E0C6E00C10BF099EC07F0AA
:101F000000C155F500C156F5EAEF0FF004014C0E83
:101F1000826F69EC0AF00401540E826F69EC0AF0DA
:101F200004012C0E826F69EC0AF084C32AF185C388
:101F30002BF186C32CF187C32DF188C32EF189C301
:101F40002FF18AC330F18BC331F18DC332F18EC3CF
:101F500033F10101B0EC1DF027EC1DF00101000E82
:101F6000046F000E056F010E066F000E076F7AEC0E
:101F70001CF0210E0C6E00C10BF099EC07F0220E44
:101F80000C6E01C10BF099EC07F0230E0C6E02C130
:101F90000BF099EC07F0240E0C6E03C10BF099ECDA
:101FA00007F000C157F501C158F502C159F503C149
:101FB0005AF5EAEF0FF004014C0E826F69EC0AF05B
:101FC0000401490E826F69EC0AF004012C0E826F45
:101FD00069EC0AF0250EAFEC07F0E8CF00F1260E11
:101FE000AFEC07F0E8CF01F1270EAFEC07F0E8CF38
:101FF00002F1280EAFEC07F0E8CF03F105EC1DF07D
:1020000031EC1BF00401730E826F69EC0AF00401DD
:102010002C0E826F69EC0AF062EC1DF0290EAFEC19
:1020200007F0E8CF00F105EC1DF031EC1BF00401E6
:10203000730E826F69EC0AF004012C0E826F69EC5A
:102040000AF051C500F152C501F153C502F154C562
:1020500003F105EC1DF031EC1BF00401730E826FEF
:1020600069EC0AF004012C0E826F69EC0AF062EC54
:102070001DF056C500F105EC1DF031EC1BF004011C
:102080006D0E826F69EC0AF004012C0E826F69EC10
:102090000AF057C500F158C501F159C502F15AC5FA
:1020A00003F10FEC17F004012C0E826F69EC0AF0BB
:1020B00073EC0AF0F4EF16F083C32AF184C32BF11A
:1020C00085C32CF186C32DF187C32EF188C32FF170
:1020D00089C330F18AC331F18BC332F18CC333F140
:1020E0000101B0EC1DF027EC1DF0160E0C6E00C1C6
:1020F0000BF099EC07F0170E0C6E01C10BF099EC88
:1021000007F0180E0C6E02C10BF099EC07F0190ED7
:102110000C6E03C10BF099EC07F000C18AF101C10C
:102120008BF102C18CF103C18DF100C18EF101C1AF
:102130008FF102C190F103C191F13EEF11F083C321
:102140002AF184C32BF185C32CF186C32DF187C3FB
:102150002EF188C32FF189C330F18AC331F18BC3CB
:1021600032F18CC333F10101B0EC1DF027EC1DF00E
:1021700000C18AF101C18BF102C18CF103C18DF163
:1021800000C18EF101C18FF102C190F103C191F143
:102190003EEF11F083C32AF184C32BF185C32CF1E8
:1021A00086C32DF187C32EF188C32FF189C330F187
:1021B0008AC331F18CC332F18DC333F10101B0EC2C
:1021C0001DF027EC1DF00101000E046F000E056FDD
:1021D000010E066F000E076F7AEC1CF01A0E0C6EE3
:1021E00000C10BF099EC07F01B0E0C6E01C10BF057
:1021F00099EC07F01C0E0C6E02C10BF099EC07F085
:102200001D0E0C6E03C10BF099EC07F000C192F1AA
:1022100001C193F102C194F103C195F13EEF11F0B8
:1022200083C32AF184C32BF185C32CF186C32DF11E
:1022300087C32EF188C32FF189C330F18AC331F1EE
:102240008CC332F18DC333F10101B0EC1DF027ECEA
:102250001DF00101000E046F000E056F010E066FE8
:10226000000E076F7AEC1CF000C192F101C193F1EE
:1022700002C194F103C195F13EEF11F0160EAFECDF
:1022800007F0E8CF00F1170EAFEC07F0E8CF01F14F
:10229000180EAFEC07F0E8CF02F1190EAFEC07F023
:1022A000E8CF03F105EC1DF031EC1BF00401730ED7
:1022B000826F69EC0AF004012C0E826F69EC0AF05F
:1022C0008AC100F18BC101F18CC102F18DC103F112
:1022D00005EC1DF031EC1BF00401730E826F69EC0C
:1022E0000AF004012C0E826F69EC0AF01A0EAFECB2
:1022F00007F0E8CF00F11B0EAFEC07F0E8CF01F1DB
:102300001C0EAFEC07F0E8CF02F11D0EAFEC07F0AA
:10231000E8CF03F10FEC17F004012C0E826F69EC8B
:102320000AF092C100F193C101F194C102F195C18B
:1023300003F10FEC17F073EC0AF0F4EF16F0040160
:10234000690E826F69EC0AF004012C0E826F69EC51
:102350000AF00101040E006F000E016F000E026F03
:10236000000E036F05EC1DF02CC182F40401300E49
:10237000822769EC0AF02DC182F40401300E822715
:1023800069EC0AF02EC182F40401300E822769EC58
:102390000AF02FC182F40401300E822769EC0AF0A2
:1023A00030C182F40401300E822769EC0AF031C199
:1023B00082F40401300E822769EC0AF032C182F403
:1023C0000401300E822769EC0AF033C182F4040163
:1023D000300E822769EC0AF004012C0E826F69EC42
:1023E0000AF00101060E006F000E016F000E026F71
:1023F000000E036F05EC1DF02CC182F40401300EB9
:10240000822769EC0AF02DC182F40401300E822784
:1024100069EC0AF02EC182F40401300E822769ECC7
:102420000AF02FC182F40401300E822769EC0AF011
:1024300030C182F40401300E822769EC0AF031C108
:1024400082F40401300E822769EC0AF032C182F472
:102450000401300E822769EC0AF033C182F40401D2
:10246000300E822769EC0AF004012C0E826F69ECB1
:102470000AF00101190E006F000E016F000E026FCD
:10248000000E036F05EC1DF02CC182F40401300E28
:10249000822769EC0AF02DC182F40401300E8227F4
:1024A00069EC0AF02EC182F40401300E822769EC37
:1024B0000AF02FC182F40401300E822769EC0AF081
:1024C00030C182F40401300E822769EC0AF031C178
:1024D00082F40401300E822769EC0AF032C182F4E2
:1024E0000401300E822769EC0AF033C182F4040142
:1024F000300E822769EC0AF004012C0E826F69EC21
:102500000AF0200EF86EF76AF66A04010900F5CFAA
:1025100082F469EC0AF00900F5CF82F469EC0AF064
:102520000900F5CF82F469EC0AF00900F5CF82F4D6
:1025300069EC0AF00900F5CF82F469EC0AF00900B1
:10254000F5CF82F469EC0AF00900F5CF82F469EC6A
:102550000AF00900F5CF82F469EC0AF073EC0AF096
:10256000F4EF16F08351630AD8A4F4EF16F0845107
:10257000610AD8A4F4EF16F085516C0AD8A4F4EFE0
:1025800016F08651410A42E08651440A1BE086510A
:10259000420AD8B419EF13F08651350AD8B47EEF49
:1025A00018F08651360AD8B4D3EF18F08651370A9E
:1025B000D8B43CEF19F08651380AD8B49AEF19F024
:1025C000F4EF16F00798079A04017A0E826F69EC0F
:1025D0000AF00401780E826F69EC0AF00401640EBF
:1025E000826F69EC0AF081A8FDEF12F00401550E2C
:1025F000826F69EC0AF002EF13F004014C0E826F57
:1026000069EC0AF073EC0AF0F4EF16F00788079A09
:1026100004017A0E826F69EC0AF00401410E826FA8
:1026200069EC0AF00401610E826F69EC0AF0F3EFC5
:1026300012F00798078A04017A0E826F69EC0AF09B
:102640000401420E826F69EC0AF00401610E826F90
:1026500069EC0AF0F3EF12F00101666737EF13F04F
:10266000676737EF13F0686737EF13F069674FEF6D
:1026700013F04F6743EF13F0506743EF13F05167C8
:1026800043EF13F052674FEF13F00101000E006F9C
:10269000000E016F000E026F000E036F12000101A9
:1026A000620E046F010E056F000E066F000E076FBD
:1026B00066C100F167C101F168C102F169C103F1AE
:1026C0006BEC1CF003BFD3EF13F00101000E046F9D
:1026D000A80E056F550E066F020E076F66C100F15A
:1026E00067C101F168C102F169C103F166C186F1F8
:1026F00067C187F168C188F169C189F16BEC1CF091
:1027000003BF8CEF13F00101000E866FA80E876FD8
:10271000550E886F020E896F0E0EAFEC07F0E8CFF2
:1027200018F10F0EAFEC07F0E8CF19F1100EAFEC77
:1027300007F0E8CF1AF1110EAFEC07F0E8CF1BF16C
:10274000B4EC1BF086C104F187C105F188C106F124
:1027500089C107F16BEC1CF0078278EC1BF0B4EC3C
:102760001BF0079278EC1BF086C100F187C101F1E4
:1027700088C102F189C103F1079278EC1BF0CC0EFD
:10278000046FE00E056F870E066F050E076F6BEC8A
:102790001CF000C118F101C119F102C11AF103C105
:1027A0001BF10BEF14F00101800E006F1A0E016F88
:1027B000060E026F000E036F4FC104F150C105F108
:1027C00051C106F152C107F16BEC1CF003AFECEF05
:1027D00013F062EC1DF012000E0EAFEC07F0E8CF24
:1027E00018F10F0EAFEC07F0E8CF19F1100EAFECB7
:1027F00007F0E8CF1AF1110EAFEC07F0E8CF1BF1AC
:102800004FC100F150C101F151C102F152C103F1B8
:10281000078278EC1BF018C100F119C101F11AC14F
:1028200002F11BC103F112000401730E826F69EC07
:102830000AF004012C0E826F69EC0AF0078462C171
:1028400066F163C167F164C168F165C169F14BC1AB
:102850004FF14CC150F14DC151F14EC152F157C130
:1028600059F158C15AF107943AEC14F073EC0AF09C
:10287000F4EF16F066C100F167C101F168C102F121
:1028800069C103F1010105EC1DF031EC1BF00401FD
:10289000630E826F69EC0AF004012C0E826F69EC02
:1028A0000AF04FC100F150C101F151C102F152C112
:1028B00003F1010105EC1DF031EC1BF00401660E83
:1028C000826F69EC0AF004012C0E826F69EC0AF049
:1028D00062EC1DF059C100F15AC101F1010105EC92
:1028E0001DF031EC1BF00401740E826F69EC0AF0EC
:1028F00012000F820401530E826F69EC0AF004018A
:102900002C0E826F69EC0AF083C32AF184C32BF189
:1029100085C32CF186C32DF187C32EF188C32FF117
:1029200089C330F18AC331F18BC332F18CC333F1E7
:102930000101B0EC1DF027EC1DF000C166F101C1F2
:1029400067F102C168F103C169F18EC32AF18FC337
:102950002BF190C32CF191C32DF192C32EF193C3AF
:102960002FF194C330F195C331F196C332F197C37F
:1029700033F10101B0EC1DF027EC1DF000C14FF167
:1029800001C150F102C151F103C152F1A3EC1DF09C
:1029900099C32FF19AC330F19BC331F19CC332F13B
:1029A0009DC333F10101B0EC1DF027EC1DF000C117
:1029B00059F101C15AF13AEC14F004012C0E826F66
:1029C00069EC0AF0EBEF14F08251520A03E10E8237
:1029D000EBEF14F00E928251750A03E10F84F2EFCF
:1029E00014F00F948251550A03E10F86F9EF14F0A9
:1029F0000F9607840FB256EF15F00FA442EF15F0B3
:102A0000B6C166F1B7C167F1B8C168F1B9C169F182
:102A1000BAC16AF1BBC16BF1BCC16CF1BDC16DF152
:102A2000BEC16EF1BFC16FF1C0C170F1C1C171F122
:102A3000C2C172F1C3C173F1C4C174F1C5C175F1F2
:102A4000C6C176F1C7C177F1C8C178F1C9C179F1C2
:102A5000CAC17AF1CBC17BF1CCC17CF1CDC17DF192
:102A6000CEC17EF1CFC17FF1D0C180F1D1C181F162
:102A7000D2C182F1D3C183F1D4C184F1D5C185F132
:102A80004AEF15F062C166F163C167F164C168F194
:102A900065C169F14BC14FF14CC150F14DC151F1CC
:102AA0004EC152F157C159F158C15AF107940EA0C5
:102AB00078EF15F00101926765EF15F0936765EF08
:102AC00015F0946765EF15F0956769EF15F078EFED
:102AD00015F02CEC13F092C104F193C105F194C1EF
:102AE00006F195C107F16BEC1CF003BFBCEF16F0CB
:102AF0002CEC13F00101000E046F000E056F010EA7
:102B0000066F000E076F99EC1CF00FA48FEF15F005
:102B10000401750E826F69EC0AF094EF15F0040160
:102B2000720E826F69EC0AF004012C0E826F69EC60
:102B30000AF005EC1DF02967A3EF15F00401200E43
:102B4000826FA6EF15F004012D0E826F69EC0AF07A
:102B500030C182F40401300E822769EC0AF031C1E1
:102B600082F40401300E822769EC0AF004012E0E73
:102B7000826F69EC0AF032C182F40401300E8227C0
:102B800069EC0AF033C182F40401300E822769EC4B
:102B90000AF004016D0E826F69EC0AF004012C0E3C
:102BA000826F69EC0AF04FC100F150C101F151C1CF
:102BB00002F152C103F1010105EC1DF031EC1BF0F3
:102BC0000401480E826F69EC0AF004017A0E826FEC
:102BD00069EC0AF004012C0E826F69EC0AF066C100
:102BE00000F167C101F168C102F169C103F101019E
:102BF00005EC1DF031EC1BF00401630E826F69ECF3
:102C00000AF004012C0E826F69EC0AF066C100F133
:102C100067C101F168C102F169C103F101010A0E46
:102C2000046F000E056F000E066F000E076F7AEC42
:102C30001CF0000E046F120E056F000E066F000EE2
:102C4000076F99EC1CF005EC1DF02AC182F4040119
:102C5000300E822769EC0AF02BC182F40401300E99
:102C6000822769EC0AF02CC182F40401300E82271D
:102C700069EC0AF02DC182F40401300E822769EC60
:102C80000AF02EC182F40401300E822769EC0AF0AA
:102C90002FC182F40401300E822769EC0AF030C1A2
:102CA00082F40401300E822769EC0AF004012E0E32
:102CB000826F69EC0AF031C182F40401300E822780
:102CC00069EC0AF032C182F40401300E822769EC0B
:102CD0000AF033C182F40401300E822769EC0AF055
:102CE0000401730E826F69EC0AF004012C0E826FEE
:102CF00069EC0AF062EC1DF059C100F15AC101F112
:102D00001EEC18F00EB288EF16F00EA0BAEF16F017
:102D100004012C0E826F69EC0AF0200EF86EF76A3F
:102D2000F66A04010900F5CF82F469EC0AF00900A3
:102D3000F5CF82F469EC0AF00900F5CF82F469EC72
:102D40000AF00900F5CF82F469EC0AF00900F5CF2A
:102D500082F469EC0AF00900F5CF82F469EC0AF01C
:102D60000900F5CF82F469EC0AF00900F5CF82F48E
:102D700069EC0AF073EC0AF00E90F4EF16F004011F
:102D8000630E826F69EC0AF004012C0E826F69EC0D
:102D90000AF0FAEC16F004012C0E826F69EC0AF0CE
:102DA0006DEC17F004012C0E826F69EC0AF0E9EC6F
:102DB00017F004012C0E826F69EC0AF00101F80E85
:102DC000006FCD0E016F660E026F030E036F0FECE6
:102DD00017F004012C0E826F69EC0AF0FFEC17F07B
:102DE00073EC0AF0F4EF16F00301A26B07900F9258
:102DF00003EF1AF0D8900E0EAFEC07F0E8CF00F119
:102E00000F0EAFEC07F0E8CF01F1100EAFEC07F0BA
:102E1000E8CF02F1110EAFEC07F0E8CF03F10101AA
:102E2000000E046F000E056F010E066F000E076F97
:102E300099EC1CF005EC1DF02AC182F40401300E5F
:102E4000822769EC0AF02BC182F40401300E82273C
:102E500069EC0AF02CC182F40401300E822769EC7F
:102E60000AF02DC182F40401300E822769EC0AF0C9
:102E70002EC182F40401300E822769EC0AF02FC1C2
:102E800082F40401300E822769EC0AF030C182F42A
:102E90000401300E822769EC0AF031C182F404018A
:102EA000300E822769EC0AF004012E0E826F69EC65
:102EB0000AF032C182F40401300E822769EC0AF074
:102EC00033C182F40401300E822769EC0AF0040158
:102ED0006D0E826F69EC0AF01200120EAFEC07F073
:102EE000E8CF00F1130EAFEC07F0E8CF01F1140EBC
:102EF000AFEC07F0E8CF02F1150EAFEC07F0E8CF2A
:102F000003F101010A0E046F000E056F000E066F3B
:102F1000000E076F7AEC1CF0000E046F120E056FA6
:102F2000000E066F000E076F99EC1CF005EC1DF00B
:102F30002AC182F40401300E822769EC0AF02BC109
:102F400082F40401300E822769EC0AF02CC182F46D
:102F50000401300E822769EC0AF02DC182F40401CD
:102F6000300E822769EC0AF02EC182F40401300E83
:102F7000822769EC0AF02FC182F40401300E822707
:102F800069EC0AF030C182F40401300E822769EC4A
:102F90000AF004012E0E826F69EC0AF031C182F44E
:102FA0000401300E822769EC0AF032C182F4040178
:102FB000300E822769EC0AF033C182F40401300E2E
:102FC000822769EC0AF00401730E826F69EC0AF043
:102FD00012000A0EAFEC07F0E8CF00F10B0EAFECD9
:102FE00007F0E8CF01F10C0EAFEC07F0E8CF02F1EB
:102FF0000D0EAFEC07F0E8CF03F11EEF18F0060E50
:10300000AFEC07F0E8CF00F1070EAFEC07F0E8CF28
:1030100001F1080EAFEC07F0E8CF02F1090EAFECBA
:1030200007F0E8CF03F11EEF18F0010162EC1DF08C
:10303000078457C100F158C101F107940101E80E5E
:10304000046F800E056F000E066F000E076F7AEC9E
:103050001CF0000E046F040E056F000E066F000ECC
:10306000076F99EC1CF0880E046F130E056F000EAD
:10307000066F000E076F6BEC1CF00A0E046F000E5B
:10308000056F000E066F000E076F99EC1CF005EC43
:103090001DF00101296752EF18F00401200E826F24
:1030A00055EF18F004012D0E826F69EC0AF030C163
:1030B00082F40401300E822769EC0AF031C182F4F7
:1030C0000401300E822769EC0AF032C182F4040157
:1030D000300E822769EC0AF004012E0E826F69EC33
:1030E0000AF033C182F40401300E822769EC0AF041
:1030F0000401430E826F69EC0AF0120087C32AF1C3
:1031000088C32BF189C32CF18AC32DF18BC32EF117
:103110008CC32FF18DC330F18EC331F190C332F1E6
:1031200091C333F10101296BB0EC1DF027EC1DF0C8
:103130000101000E046F000E056F010E066F000EF8
:10314000076F7AEC1CF00E0E0C6E00C10BF099ECC0
:1031500007F00F0E0C6E01C10BF099EC07F0100E8A
:103160000C6E02C10BF099EC07F0110E0C6E03C14E
:103170000BF099EC07F004017A0E826F69EC0AF00B
:1031800004012C0E826F69EC0AF00401350E826F87
:1031900069EC0AF004012C0E826F69EC0AF0FAEC7B
:1031A00016F002EF13F087C32AF188C32BF189C30D
:1031B0002CF18AC32DF18BC32EF18CC32FF18DC35B
:1031C00030F18EC331F190C332F191C333F101017B
:1031D000296BB0EC1DF027EC1DF0880E046F130E68
:1031E000056F000E066F000E076F6FEC1CF0000EEF
:1031F000046F040E056F000E066F000E076F7AEC69
:103200001CF00101E80E046F800E056F000E066FC2
:10321000000E076F99EC1CF00A0E0C6E00C10BF04B
:1032200099EC07F00B0E0C6E01C10BF099EC07F056
:103230000C0E0C6E02C10BF099EC07F00D0E0C6E2B
:1032400003C10BF099EC07F004017A0E826F69EC70
:103250000AF004012C0E826F69EC0AF00401360EAC
:10326000826F69EC0AF004012C0E826F69EC0AF09F
:10327000E9EC17F002EF13F087C32AF188C32BF1B2
:1032800089C32CF18AC32DF18BC32EF18CC32FF18E
:103290008DC330F18FC331F190C332F191C333F15B
:1032A0000101B0EC1DF027EC1DF0000E046F120EB2
:1032B000056F000E066F000E076F7AEC1CF001011F
:1032C0000A0E046F000E056F000E066F000E076FEA
:1032D00099EC1CF0120E0C6E00C10BF099EC07F08B
:1032E000130E0C6E01C10BF099EC07F0140E0C6E6E
:1032F00002C10BF099EC07F0150E0C6E03C10BF038
:1033000099EC07F004017A0E826F69EC0AF004016F
:103310002C0E826F69EC0AF00401370E826F69ECA3
:103320000AF004012C0E826F69EC0AF06DEC17F0C4
:1033300002EF13F087C32AF188C32BF189C32CF164
:103340008AC32DF18BC32EF18CC32FF18DC330F1C5
:103350008EC331F190C332F191C333F10101296B76
:10336000B0EC1DF027EC1DF0880E046F130E056FF6
:10337000000E066F000E076F6FEC1CF0000E046F5E
:10338000040E056F000E066F000E076F7AEC1CF03E
:103390000101E80E046F800E056F000E066F000E2F
:1033A000076F99EC1CF0060E0C6E00C10BF099EC47
:1033B00007F0070E0C6E01C10BF099EC07F0080E38
:1033C0000C6E02C10BF099EC07F0090E0C6E03C1F4
:1033D0000BF099EC07F004017A0E826F69EC0AF0A9
:1033E00004012C0E826F69EC0AF00401380E826F22
:1033F00069EC0AF004012C0E826F69EC0AF0FFEC14
:1034000017F002EF13F081A8C1EF1AF007A87AEFC6
:103410001AF00101800E006F1A0E016F060E026F86
:10342000000E036F4BC104F14CC105F14DC106F113
:103430004EC107F16BEC1CF003BFC1EF1AF02BEC8F
:103440001BF04BC100F14CC101F14DC102F14EC165
:1034500003F1078278EC1BF018C104F119C105F1E2
:103460001AC106F11BC107F1F80E006FCD0E016FF6
:10347000660E026F030E036F6BEC1CF00E0E0C6EEB
:1034800000C10BF099EC07F00F0E0C6E01C10BF0B0
:1034900099EC07F0100E0C6E02C10BF099EC07F0DE
:1034A000110E0C6E03C10BF099EC07F007840101BB
:1034B00062EC1DF057C100F158C101F107940A0EEA
:1034C0000C6E00C10BF099EC07F00B0E0C6E01C1F5
:1034D0000BF099EC07F00C0E0C6E02C10BF099EC9E
:1034E00007F00D0E0C6E03C10BF099EC07F0079876
:1034F000C1EF1AF007AAC1EF1AF00784010162ECCC
:103500001DF057C100F158C101F10794060E0C6E71
:1035100000C10BF099EC07F0070E0C6E01C10BF027
:1035200099EC07F0080E0C6E02C10BF099EC07F055
:10353000090E0C6E03C10BF099EC07F0078462C111
:1035400000F163C101F164C102F165C103F10794A7
:10355000120E0C6E00C10BF099EC07F0130E0C6EFE
:1035600001C10BF099EC07F0140E0C6E02C10BF0C8
:1035700099EC07F0150E0C6E03C10BF099EC07F0F7
:10358000079A0401805181197F0B0BE09EA809D096
:1035900014EE00F081517F0BE126E750812B0F01E3
:1035A000AD6E05012951010A13E081AAE8EF1AF076
:1035B00005012951000A0AE00EB8E8EF1AF00501EA
:1035C0002A67E8EF1AF00EB8E8EF1AF0A5EF23F03B
:1035D00081B8FDEF1AF07FEC1EF005012951020AB7
:1035E00002E0FDEF1AF0562FFDEF1AF055C556F523
:1035F0000501010E2A6F3C0E2B6FD7EF09F018C1A1
:1036000000F119C101F11AC102F11BC103F1000E51
:10361000046F000E056F010E066F000E076F99EC28
:103620001CF029A12AEF1BF02051D8B42AEF1BF07F
:1036300018C100F119C101F11AC102F11BC103F156
:10364000000E046F000E056F0A0E066F000E076F66
:1036500099EC1CF012000101186B196B1A6B1B6BB3
:1036600012002AC182F40401300E822769EC0AF0AC
:103670002BC182F40401300E822769EC0AF02CC1C0
:1036800082F40401300E822769EC0AF02DC182F425
:103690000401300E822769EC0AF02EC182F4040185
:1036A000300E822769EC0AF02FC182F40401300E3B
:1036B000822769EC0AF030C182F40401300E8227BF
:1036C00069EC0AF031C182F40401300E822769EC02
:1036D0000AF032C182F40401300E822769EC0AF04C
:1036E00033C182F40401300E822769EC0AF0120023
:1036F0000101005305E1015303E1025301E1002BF5
:103700003BEC1CF062EC1DF03951006F3A51016F37
:10371000420E046F4B0E056F000E066F000E076F12
:103720007AEC1CF000C104F101C105F102C106F1FF
:1037300003C107F118C100F119C101F11AC102F169
:103740001BC103F107B2A9EF1BF06FEC1CF0ABEF4C
:103750001BF06BEC1CF000C118F101C119F102C1A2
:103760001AF103C11BF1120062EC1DF059C100F106
:103770005AC101F1060EAFEC07F0E8CF04F1070ED5
:10378000AFEC07F0E8CF05F1080EAFEC07F0E8CF9B
:1037900006F1090EAFEC07F0E8CF07F16BEC1CF077
:1037A00000C124F101C125F102C126F103C127F1B5
:1037B000290E046F000E056F000E066F000E076FD6
:1037C0007AEC1CF0EE0E046F430E056F000E066FD0
:1037D000000E076F6FEC1CF024C104F125C105F148
:1037E00026C106F127C107F17AEC1CF000C11CF1DB
:1037F00001C11DF102C11EF103C11FF1120EAFEC98
:1038000007F0E8CF04F1130EAFEC07F0E8CF05F1B5
:10381000140EAFEC07F0E8CF06F1150EAFEC07F091
:10382000E8CF07F10D0E006F000E016F000E026F62
:10383000000E036F7AEC1CF0180E046F000E056F7B
:10384000000E066F000E076F99EC1CF01CC104F10E
:103850001DC105F11EC106F11FC107F16FEC1CF07F
:103860006A0E046F2A0E056F000E066F000E076FBA
:103870006BEC1CF01200BF0EFA6E200E3A6F396B23
:10388000D8900037013702370337D8B04CEF1CF01F
:103890003A2F41EF1CF039073A070353D8B412000E
:1038A0000331070B80093F6F03390F0B010F396F8D
:1038B00080EC5FF0406F390580EC5FF0405D405F69
:1038C000396B3F33D8B0392739333FA961EF1CF04A
:1038D00040513927120087EC1DF0D8B01200035177
:1038E0000719346F4AEC1DF0D8900751031934AF13
:1038F000800F1200346B6EEC1DF0D8A084EC1DF02C
:10390000D8B0120059EC1DF062EC1DF01F0E366F9E
:103910009AEC1DF00B35D8B04AEC1DF0D8A0033559
:10392000D8B01200362F88EF1CF034B171EC1DF0C6
:103930001200346B04510511061107110008D8A0BC
:103940006EEC1DF0D8A084EC1DF0D8B01200086B0E
:10395000096B0A6B0B6B9AEC1DF01F0E366F9AEC1D
:103960001DF007510B5DD8A4C2EF1CF006510A5D93
:10397000D8A4C2EF1CF00551095DD8A4C2EF1CF019
:103980000451085DD8A0D5EF1CF00451085F055123
:10399000D8A0053D095F0651D8A0063D0A5F075132
:1039A000D8A0073D0B5FD8900081362FAFEF1CF0F9
:1039B00034B171EC1DF0346B6EEC1DF0D8909EECC0
:1039C0001DF007510B5DD8A4F2EF1CF006510A5D03
:1039D000D8A4F2EF1CF00551095DD8A4F2EF1CF059
:1039E0000451085DD8A001EF1DF0003F01EF1DF06C
:1039F000013F01EF1DF0023F01EF1DF0032BD8B492
:103A0000120034B171EC1DF012000101346B6EEC48
:103A10001DF0D8B01200A3EC1DF0200E366F003759
:103A200001370237033711EE33F00A0E376FE736EE
:103A30000A0EE75CD8B0E76EE552372F17EF1DF09E
:103A4000362F0FEF1DF034B12981D89012000101FB
:103A50000A0E346F200E366F11EE29F03451376F95
:103A60000A0ED890E652D8B0E726E732372F32EF69
:103A70001DF00333023301330033362F2CEF1DF0DA
:103A8000E750FF0FD8A00335D8B0120029B171EC70
:103A90001DF01200045100270551D8B0053D012743
:103AA0000651D8B0063D02270751D8B0073D03277D
:103AB00012000051086F0151096F02510A6F035142
:103AC0000B6F12000101006B016B026B036B1200A4
:103AD0000101046B056B066B076B12000335D8A060
:103AE00012000351800B001F011F021F031F003F24
:103AF00081EF1DF0013F81EF1DF0023F81EF1DF0CE
:103B0000032B342B032512000735D8A012000751D0
:103B1000800B041F051F061F071F043F97EF1DF0B2
:103B2000053F97EF1DF0063F97EF1DF0072B342B55
:103B300007251200003701370237033708370937E6
:103B40000A370B3712000101296B2A6B2B6B2C6B88
:103B50002D6B2E6B2F6B306B316B326B336B120016
:103B60002A510F0B2A6F2B510F0B2B6F2C510F0B60
:103B70002C6F2D510F0B2D6F2E510F0B2E6F2F51C0
:103B80000F0B2F6F30510F0B306F31510F0B316F07
:103B900032510F0B326F33510F0B336F1200898488
:103BA000000EC76E220EC66E9E96C69E000EC96E91
:103BB000FF0E9EB602D0E82EFCD79E96C69E000E43
:103BC000C96EFF0E9EB602D0E82EFCD7C9CFA5F570
:103BD0009E96C69E000EC96EFF0E9EB602D0E82EBF
:103BE000FCD7C9CFA6F59E96C69E000EC96EFF0EE5
:103BF0009EB602D0E82EFCD7C9CFA7F59E96C69EEA
:103C0000000EC96EFF0E9EB602D0E82EFCD7C9CFBB
:103C1000A8F59E96C69E000EC96EFF0E9EB602D0F7
:103C2000E82EFCD7C9CFA9F59E96C69E000EC96E98
:103C3000FF0E9EB602D0E82EFCD7C9CFAAF59E96FD
:103C4000C69E000EC96EFF0E9EB602D0E82EFCD7AF
:103C5000C9CFABF5899482EC20F012008984000E64
:103C6000C76E220EC66E9E96C69E800EC96EFF0E51
:103C70009EB602D0E82EFCD79E96C69EA5C5C9FF6B
:103C8000FF0E9EB602D0E82EFCD79E96C69EA6C515
:103C9000C9FFFF0E9EB602D0E82EFCD79E96C69EA8
:103CA000A7C5C9FFFF0E9EB602D0E82EFCD79E9690
:103CB000C69EA8C5C9FFFF0E9EB602D0E82EFCD74F
:103CC0009E96C69EA9C5C9FFFF0E9EB602D0E82EDD
:103CD000FCD79E96C69EAAC5C9FFFF0E9EB602D00F
:103CE000E82EFCD79E96C69EABC5C9FFFF0E9EB6BA
:103CF00002D0E82EFCD7899482EC20F0120089844F
:103D0000000EC76E220EC66E9E96C69E070EC96E28
:103D1000FF0E9EB602D0E82EFCD79E96C69E000EE1
:103D2000C96EFF0E9EB602D0E82EFCD7C9CFA5F50E
:103D30009E96C69E000EC96EFF0E9EB602D0E82E5D
:103D4000FCD7C9CFA6F59E96C69E000EC96EFF0E83
:103D50009EB602D0E82EFCD7C9CFA7F59E96C69E88
:103D6000000EC96EFF0E9EB602D0E82EFCD7C9CF5A
:103D7000A8F5899482EC20F08984000EC76E220E8B
:103D8000C66E9E96C69E0F0EC96EFF0E9EB602D0E0
:103D9000E82EFCD79E96C69E000EC96EFF0E9EB6FC
:103DA00002D0E82EFCD7C9CFADF5899482EC20F083
:103DB00012008984000EC76E220EC66E9E96C69EA5
:103DC000870EC96EFF0E9EB602D0E82EFCD79E96D7
:103DD000C69EA5C5C9FFFF0E9EB602D0E82EFCD731
:103DE0009E96C69EA6C5C9FFFF0E9EB602D0E82EBF
:103DF000FCD79E96C69EA7C5C9FFFF0E9EB602D0F1
:103E0000E82EFCD79E96C69EA8C5C9FFFF0E9EB69B
:103E100002D0E82EFCD7899482EC20F089849E960B
:103E2000C69E8F0EC96EFF0E9EB602D0E82EFCD73E
:103E30009E96C69EADC5C9FFFF0E9EB602D0E82E67
:103E4000FCD7899482EC20F012008984000EC76EA2
:103E5000220EC66E9E96C69E870EC96EFF0E9EB639
:103E600002D0E82EFCD79E96C69E000EC96EFF0EAD
:103E70009EB602D0E82EFCD79E96C69E800EC96ED6
:103E8000FF0E9EB602D0E82EFCD79E96C69E800EF0
:103E9000C96EFF0E9EB602D0E82EFCD79E96C69E37
:103EA000800EC96EFF0E9EB602D0E82EFCD7899414
:103EB00082EC20F089849E96C69E8F0EC96EFF0EFE
:103EC0009EB602D0E82EFCD79E96C69E010EC96E05
:103ED000FF0E9EB602D0E82EFCD7899482EC20F02B
:103EE00012008984000EC76E220EC66E9E96C69E74
:103EF000870EC96EFF0E9EB602D0E82EFCD79E96A6
:103F0000C69E000EC96EFF0E9EB602D0E82EFCD7EC
:103F10009E96C69E000EC96EFF0E9EB602D0E82E7B
:103F2000FCD79E96C69E800EC96EFF0E9EB602D02E
:103F3000E82EFCD79E96C69E800EC96EFF0E9EB6DA
:103F400002D0E82EFCD7899482EC20F089849E96DA
:103F5000C69E8F0EC96EFF0E9EB602D0E82EFCD70D
:103F60009E96C69E010EC96EFF0E9EB602D0E82E2A
:103F7000FCD7899482EC20F012008984000EC76E71
:103F8000220EC66E9E96C69E8F0EC96EFF0E9EB600
:103F900002D0E82EFCD782EC20F09E96C69E810EC1
:103FA000C96EFF0E9EB602D0E82EFCD7899482EC33
:103FB00020F08984000EC76E220EC66E9E96C69EA5
:103FC0008F0EC96EFF0E9EB602D0E82EFCD782EC93
:103FD00020F09E96C69E010EC96EFF0E9EB602D0C0
:103FE000E82EFCD7899482EC20F089849E96C69EA8
:103FF000910EC96EFF0E9EB602D0E82EFCD782EC61
:1040000020F09E96C69EA50EC96EFF0E9EB602D0EB
:10401000E82EFCD7899482EC20F012008984000EEF
:10402000C76E220EC66E9E96C69E8F0EC96EFF0E7E
:104030009EB602D0E82EFCD782EC20F09E96C69E5B
:10404000810EC96EFF0E9EB602D0E82EFCD7899471
:1040500082EC20F012008984000EC76E220EC66E1C
:104060009E96C69E8F0EC96EFF0E9EB602D0E82E9B
:10407000FCD782EC20F09E96C69E010EC96EFF0E04
:104080009EB602D0E82EFCD7899482EC20F0120074
:104090008984000EC76E220EC66E9E96C69E910E35
:1040A000C96EFF0E9EB602D0E82EFCD782EC20F03F
:1040B0009E96C69EA50EC96EFF0E9EB602D0E82E35
:1040C000FCD7899482EC20F012008984000EC76E20
:1040D000220EC66E9E96C69E910EC96EFF0E9EB6AD
:1040E00002D0E82EFCD782EC20F09E96C69E000EF1
:1040F000C96EFF0E9EB602D0E82EFCD7899482ECE2
:1041000020F01200050EE82EFED71200200EC66E1B
:104110000501256B266B276B286B899A400EC76EAD
:10412000200EC66E9E96C69E030EC96EFF0E9EB6EC
:1041300002D0E82EFCD79E96C69E27C5C9FFFF0E6B
:104140009EB602D0E82EFCD79E96C69E26C5C9FF15
:10415000FF0E9EB602D0E82EFCD79E96C69E25C5C1
:10416000C9FFFF0E9EB602D0E82EFCD79E96C69ED3
:10417000C952FF0E9EB602D0E82EFCD7898AC950DC
:10418000FF0A02E1CDEF20F0100E2527E86A262372
:10419000E86A272327A98DEF20F0220EC66E1200B1
:1041A000899A400EC76E200EC66E9E96C69E060E5B
:1041B000C96EFF0E9EB602D0E82EFCD7898A899A76
:1041C0009E96C69EC70EC96EFF0E9EB602D0E82E02
:1041D000FCD7898A899A9E96C69E050EC96EFF0EE7
:1041E0009EB602D0E82EFCD79E96C69EC952FF0E00
:1041F0009EB602D0E82EFCD7C9B0F4EF20F0898A31
:104200000501256B266B276B286B12000501FE0E3E
:104210002D6F0501000E2D6FCFEC1DF0A5C52EF5FD
:10422000A6C52FF5A7C530F5A8C531F5A9C532F546
:10423000AAC533F5ABC534F50784B6C166F1B7C17D
:1042400067F1B8C168F1B9C169F14BC14FF14CC117
:1042500050F14DC151F14EC152F157C159F158C100
:104260005AF107942CEC13F000C135F501C136F575
:1042700002C137F503C138F50501576747EF21F053
:10428000586747EF21F0596747EF21F05A674BEF26
:1042900021F059EF21F057C504F158C505F159C572
:1042A00006F15AC507F101016BEC1CF003BFC7EF23
:1042B00021F059C139F55AC13AF5AFC53BF5B0C542
:1042C0003CF50501100E2C6F899A400EC76E200E2A
:1042D000C66E9E96C69E060EC96EFF0E9EB602D094
:1042E000E82EFCD7898A899A9E96C69E020EC96ED0
:1042F000FF0E9EB602D0E82EFCD79E96C69E27C51E
:10430000C9FFFF0E9EB602D0E82EFCD79E96C69E31
:1043100026C5C9FFFF0E9EB602D0E82EFCD79E969A
:10432000C69E25C5C9FFFF0E9EB602D0E82EFCD75B
:1043300025EE2DF02C2F02D0A9EF21F09E96C69EDF
:10434000DECFC9FFFF0E9EB602D0E82EFCD79AEF53
:1043500021F0898A899A9E96C69E050EC96EFF0E27
:104360009EB602D0E82EFCD79E96C69EC952FF0E7E
:104370009EB602D0E82EFCD7C9B0B4EF21F0898AEE
:104380000501100E2527E86A2623E86A2723120074
:1043900019C502F51AC503F525EE5FF005012C6B72
:1043A00016EE00F005010251E1260351D8B00329B1
:1043B000E226E7CFE8FF2C0A06E12CC5DEFF050167
:1043C0002C6BEBEF21F0E7CFE8FF2A0A0CE0E7CFF8
:1043D000DEFF05012C2B0501032B023F0307030E13
:1043E0000317D0EF21F005012D6B2E6B2F6B306B77
:1043F000316B326B336B346B356B366B376B386BC1
:10440000396B3A6B3B6B3C6B3D6B3E6B3F6B406B70
:10441000416B426B436B446B456B466B476B486B20
:10442000496B4A6B4B6B4C6BDDCFE8FF05012C51A0
:1044300005E0DDCFE8FF2C2F19EF22F00501DDCFDD
:104440002CF52C5105E0DDCFE8FF2C2F23EF22F0D7
:104450000501DDCF2CF52C5105E0DDCFE8FF2C2F39
:104460002DEF22F011EE33F00101A3EC1DF0050158
:10447000DDCF2CF52C5105E0DDCFE5FF2C2F3CEFF7
:1044800022F00101B0EC1DF027EC1DF000C12EF56B
:1044900001C12FF502C130F50501DDCF2CF52C51FE
:1044A00005E0DDCFE8FF2C2F51EF22F00501DDCF35
:1044B0002CF52C5105E0DDCFE8FF2C2F5BEF22F02F
:1044C0000501DDCF2CF52C5107E0DDCFE8FFE8A892
:1044D0002D852C2F65EF22F011EE33F00101A3ECB6
:1044E0001DF00501DDCF2CF52C5114E0DDCFE5FFEB
:1044F000DDCFE5FFDDCFE5FFDDCFE5FFDDCFE8FF79
:10450000DDCFE5FFDDCFE5FFDDCFE5FFDDCFE5FF6B
:10451000DDCFE5FF0101B0EC1DF027EC1DF000C17F
:1045200038F501C139F502C13AF503C13BF5050182
:10453000DDCF2CF52C5107E0DDCFE8FFE8A82D8377
:104540002C2F9CEF22F011EE33F00101A3EC1DF0B3
:104550000501DDCF2CF52C5105E0DDCFE5FF2C2F3B
:10456000ADEF22F001012EC12FF12DC12EF12CC192
:104570002DF12BC12CF1B0EC1DF027EC1DF000C18A
:1045800034F501C135F502C136F503C137F5050132
:10459000DDCF2CF52C5107E0DDCFE8FF2C2FCCEF41
:1045A00022F0E8B02D8711EE33F00101A3EC1DF0ED
:1045B000DDCFE8FFDDCFE8FFDDCFE8FFDDCFE8FFAF
:1045C000DDCFE8FFDDCFE5FFDDCFE5FFDDCFE5FFA8
:1045D000DDCFE5FFDDCFE5FFDDCFE5FFB0EC1DF082
:1045E00027EC1DF000C131F501C132F502C133F5F0
:1045F000078462C166F163C167F164C168F165C196
:1046000069F14BC14FF14CC150F14DC151F14EC157
:1046100052F157C159F158C15AF107942CEC13F0DB
:1046200000C13CF501C13DF502C13EF503C13FF5B6
:10463000120021C500F122C501F123C502F124C5F4
:1046400003F1899A400EC76E200EC66E9E96C69ED6
:104650000B0EC96EFF0E9EB602D0E82EFCD79E96BA
:10466000C69E02C1C9FFFF0E9EB602D0E82EFCD73F
:104670009E96C69E01C1C9FFFF0E9EB602D0E82ECF
:10468000FCD79E96C69E00C1C9FFFF0E9EB602D003
:10469000E82EFCD79E96C69EC952FF0E9EB602D04B
:1046A000E82EFCD725EE2DF00501100E2C6F9E96FE
:1046B000C69EC952FF0E9EB602D0E82EFCD7C9CFC7
:1046C000DEFF2C2F57EF23F0898A1200899A400EC3
:1046D000C76E200EC66E9E96C69E900EC96EFF0EC9
:1046E0009EB602D0E82EFCD79E96C69E000EC96EDE
:1046F000FF0E9EB602D0E82EFCD79E96C69E000EF8
:10470000C96EFF0E9EB602D0E82EFCD79E96C69EBE
:10471000000EC96EFF0E9EB602D0E82EFCD79E9604
:10472000C69EC952FF0E9EB602D0E82EFCD7C9CF56
:104730002DF59E96C69EC952FF0E9EB602D0E82E5B
:10474000FCD7C9CF2EF5898A12007FEC1EF0F29CAF
:10475000F29E8B948A86899CC69AC2908A94898A92
:104760009482948C720ED36ED3A4FED789968A90CD
:104770009390FF0EE8CF00F0E82EFED7002EFCD776
:104780008150F294F29A9E909D909E929D92F29802
:0C479000F292F290F286F28E0300FF001D
:10BF0000E844F926000C160C2B0C3F0C520C640C68
:10BF1000760C860C960CA50CB30CC10CCF0CDC0C6B
:06BF2000E80CF40C000C1B
:00000001FF
